:020000020000FC
:100000000BC045C178C107C006C005C004C0A6C169
:1000100002C001C000C018950FED0DBF03EE07BB75
:100020000CE108BB03E401BB00E002BB0AE005BF32
:1000300008E90AB903E3B49B0CE0B39B09E1B49966
:1000400003C0B39901C008E009B933274BE0772713
:10005000ABE088279927BB27CC27DD2701E0B02E0E
:10006000A02E00EC0BBF78949B7BEE24C19AC09A23
:1000700037D0C098C19858E04424440C0027B29B64
:1000800001E0402A2DD0C19A2BD0C1985A95A9F7EA
:1000900058E05524550C0027B29B01E0502A20D08F
:1000A000C19A1ED0C1985A95A9F71AD0042D0125DE
:1000B00019F4052D0225C9F00AE4202F86D002E0AC
:1000C000202F83D0242D040D80D0252D050D7DD02B
:1000D000252D050D7AD0202F78D0142C252C05C085
:1000E0000CE00A95F1F70895C1CF90FD07C094FD8B
:1000F00008C092FD09C096FD09C0B8CF93FDA1F7D5
:1001000007C097FD89F716C02ED0AECF25D0ACCF53
:10011000FC2C5FD009D091FF03C0FD2C5AD004D035
:100120009E7F9D7FDE7FA0CF9B7FD160EE2492FFDC
:10013000FECF0895862C7CD009D095FF03C0872C74
:1001400077D004D09F7E9F7DDD7F8ECF9F7BD26056
:10015000EE2496FFFECF08950DE4202F36D0E8E67A
:10016000F0E0908024C0E0E6F0E09080E0E6F0E08F
:10017000E90D4080E4E6F0E0E90D5080452419F4F3
:100180009A94A1F721C0E0E6F0E09080E0E6F0E08C
:10019000E90D4080E4E6F0E0E90D40829A94B1F781
:1001A000E0E6F0E090800BE4202F0FD00027292D0F
:1001B0000CD003E0902E022FE395208106D0020F91
:1001C0009A94D1F7202F01D008955D9BFECF2CB9D2
:1001D0000895F894929894988A9A00E800000A95F5
:1001E000E9F78C9A8A9868E033241DD0F79410F0D0
:1001F0008C9A02C08C98339416D06A95B9F730FC6B
:1002000002C08C9801C08C9A0ED08C980CD0849B24
:1002100003C00FEFF02EDDCF829BFECF33274BE0E4
:10022000882778940895829BFECF8299FECF089507
:10023000F894939895988B9A00E800000A95E9F74E
:100240008D9A8B9868E033241DD0879410F08D9A96
:1002500002C08D98339416D06A95B9F730FC02C06D
:100260008D9801C08D9A0ED08D980CD0859B03C0BF
:100270000FEF802EDDCF839BFECF7727ABE0882763
:1002800078940895839BFECF8399FECF08950FB68F
:100290000F921F93986082FD0CC04B3028F44330BE
:1002A00018F036958499306815B7136015BF8460CF
:1002B0001EC015B71E7F15BF8B7F4A95C1F4E32E74
:1002C00033274BE0D0FD0AC0E7FE08C0E6FE06C0BB
:1002D000E0E6F0E0EA0DE082A39409C0E0E6F0E099
:1002E000A082EA0DE082AA24A3949460977F1F91D4
:1002F0000F900FBE18950FB60F921F93906885FD53
:100300000CC0AB3028F4A33018F07695859970684E
:1003100015B71C6015BF80621DC015B71B7F15BFC8
:100320008F7DAA95B9F4E72E7727ABE0D1FD09C000
:100330001B2D133031F0E8E6F0E0EB0DE082B394D2
:1003400009C0E8E6F0E0B082EB0DE082BB24B39494
:1003500090649F771F910F900FBE18950FB60F9264
:100360001F930F931CB1CC2309F04AC01635D9F462
:1003700020E52BDF23E529DF22E327DF23E525DF47
:1003800025E423DF22E521DF20E21FDF26E51DDF54
:1003900020E31BDF2EE219DF21E317DF2EE215DF5A
:1003A00021E313DF5BC01C3421F42B2F20630DDF0E
:1003B00055C0123529F491600FEFC02EBB274EC0F7
:1003C000153411F4C8604AC01B3411F4C16046C032
:1003D0001B3611F4C26042C0123721F490610FEF56
:1003E000602E3CC0153621F4906104EF602E36C0BB
:1003F0001D3411F4C06132C01D3681F5C0622EC0BB
:10040000C3FF08C0916092600DEEC02E1770D12E10
:10041000CC2724C0C0FF04C09160C12ECC271EC0D1
:10042000C2FF05C091609260D12ECC2717C0C1FFDA
:1004300003C0C12EC46012C0C4FF04C09061612E0D
:10044000CC270CC0C6FF05C090619062712ECC27EE
:1004500005C0C5FF03C0612EC06400C00F911F918D
:060460000F900FBE18957D
:00000001FF
